:10000000E8C6000002C700000C94C214FEC600003F
:10001000FCC600000C945418F8C60000F6C6000098
:10002000F4C600000C94CE1CF0C60000EEC6000022
:10003000ECC60000EAC60000E8C60000E6C6000004
:10004000E4C60000E2C60000E0C60000DEC6000014
:10005000DCC600000C94D71ED8C60000D6C600002F
:10006000D4C60000D2C60000C00000000000B600E8
:10007000E308DD08C600CE085308CF00A3073C08FC
:10008000D500B007A808E500B8078208F200C0074D
:100090004B080001C80767080901D5072D0816019C
:1000A000E4075B082601F1071E083201FF070F086D
:1000B000000000000000456967656E652049440046
:1000C0005345545550004B6F6E7472617374004CFD
:1000D00069636874005369676E616C3A204D65739B
:1000E00073616765005369676E616C3A205573658B
:1000F000720053656E64657665727375636865003A
:100100004672657175656E7A00435120656D706643
:10011000616E67656E0042616B656E20496E746545
:100120007276616C6C005265706561742D466C610D
:1001300067004645430048415550544D454E5500D3
:100140004D48656172640056657266617373656ED1
:10015000004E6163687269636874656E004572770A
:1001600065697465727400536574757000417573C8
:10017000736368616C74656E0036010000000040B6
:1001800001E80900004701CA0900005101C6090041
:10019000005D01B90900006701BF0900006D017A27
:1001A000090000000000000000DD0100000000E781
:1001B00001280A0000D301090A0000EE01F6090037
:1001C000000002ED0900000C02EB09000000000035
:1001D000000000456D7066E46E676572005645521A
:1001E00046415353454E0053656E64656E00456E3F
:1001F00074777572662073706569636865726E00E6
:1002000054657874206C656572656E004265656E34
:1002100064656E0044657461696C73005D02000082
:10022000000046028B0A000050027B0A00006702B1
:100230006F0A00007502740A00001402710A0000BF
:10024000000000000000416E74776F7274656E00EC
:100250005765697465726C656974656E004E4143DB
:100260004852494348540045726E65757420736561
:100270006E64656E004CF6736368656E0053656E60
:1002800064656E00A202000000007D02A80A000062
:10029000A902AA0A0000B102AC0A00000000000096
:1002A00000004D4845415244004CF6736368656E4A
:1002B00000416C6C65206CF6736368656E0000012C
:1002C00008080900213C221F243E21322A25222A27
:1002D000150C083F2E2A131C2A11023A0F142A1556
:1002E000042A1D290814232214093C0A3D3E2A151C
:1002F0001C22233E221D3E2A233E0A031C223B3E93
:10030000083F223E2310201F3E08373E20213E0C8E
:100310003F3E043F1C221D3E0A051C323D3E0A356D
:100320002C2A1B023E033E203F1E201F3E183F3654
:100330000837063807322A2732283B000001BEBFA3
:100340000E000E0128FE2828FE294C9EF29EF26522
:100350000C12522C10689490616CFE92BE6CE09965
:100360000403387CC68382C67C3914083E0815080D
:10037000083E08093071101011C0C1C0300F7CFE5A
:100380008282FE7D84FEFE818CC2E2B29E8D44821A
:100390009292FE6D302824FEFE214E8E8A8AFA73D8
:1003A0007CFE9292F2610202E2FA1E076CFE9292C9
:1003B000FE6D0C9E92D27E3DEC0D6C6D3030484847
:1003C0008485282828282984844848303104A2B20A
:1003D0001E0D384492BAAA9ABA2419E0F83E263E75
:1003E000F8E1FEFE9292FE6D7CFE8282C645FEFE24
:1003F0008282FE7DFEFE929283FEFE1212037CFE3E
:100400008292F2F5FEFE101010FEFF82FEFE838047
:1004100082FE7FFEFE386CC683FEFE808081FEFE7B
:100420000E1C38180CFEFFFE0E1C3870FF7CFE827E
:100430008282FE7DFEFE22223E1D3C7E4262C2FE84
:10044000BDFEFE3272DE8D4C9EBAF2650202FEFEE9
:1004500002037EFE8080FE7F0E3EF0F03E0F3EFEE9
:10046000C03E3EC0FE3FC6EE3838EEC7061EF8F866
:100470001E07E2F2BA9E8FFEFE82830638C1828298
:10048000FEFF08040202040980808080808102054A
:1004900040E8A8F8F1FEFE88F87170F8888970F8D5
:1004A00088FEFF70F8A8B8B1FCFE0A0310B8A8F8DF
:1004B00079FEFE08F8F1FAFB88FA7BFEFE70D88917
:1004C000FEFFF8F808F8F008F8F1F8F808F8F1700D
:1004D000F888F871F8F8283811103828F8F9F8F881
:1004E000101990B8E8497CFC8978F880F8F91878F8
:1004F000E0781938F8C030C0F839D8F820F8D918A1
:10050000B8E07819C8E8B899E3F83E263EF8E77AEB
:10051000FE848484FE7B7AFA8080FA7B42EAA8FA21
:10052000F372FA88FA737AFA80FAFBFC7E92FE6D17
:10053000000001BF0E000F20E83E28F82E09889425
:10054000FEA4454626100864636C92926C508104A8
:10055000020138448382443914083E081508083ED5
:100560000809C1202141C038077C82827D84FE8138
:10057000C2A2928D8292926D302824FE219E929288
:10058000637C92926182621A076C92926D0C9292D5
:100590007D8069D92050505089505050505051881A
:1005A0005050502102A2120D384492AABA2419E0E8
:1005B000382638E1FE92926D7C82828245FE8282EC
:1005C0004439FE929283FE1212037C829292F5FECF
:1005D00010101010FF82FE8380827FFE102844835B
:1005E000FE808081FE0618601806FFFE04081020B9
:1005F000FF38448282824439FE2222221D384482FE
:10060000A242C4B9FE1232528D8C929292630202BF
:10061000FE02037E808080807F0E30C0C0300F3E9F
:10062000C0380638C03FC6281028C70618E018078B
:10063000C2B28A87FE830638C182FF080402040919
:100640008080808081020540A8A8F1FE88887170B2
:100650008889708888FF70A8A8B1FC121310A8A818
:1006600079FE0808F1FB887BFE205089FFF8080816
:10067000F00808F1F80808F170888871F828281146
:10068000102828F9F8100990A8497C89788080F909
:10069000186080601938C0601860C039D820D91837
:1006A000A0A079C8A899E2382638E33A4482828229
:1006B000443B7A808080807B40AAA8F3728888734C
:1006C0007A8080FBFC02926D3B033005BE023E0344
:1006D00033050000400334050000440337050000E3
:1006E0004A033E0500005003430500005903490535
:1006F000000060034F05000062035205000066031E
:10070000550500006A03580500006F035D050000F1
:1007100074036205000076036305C0027903650572
:10072000C3027B03660500007E036905C5028403DE
:100730006D05C80288037005CB028E037405CE02D6
:1007400094037805D1029A037D05D402A0038105A4
:10075000D702A6038505DA02AC038905DD02B203E0
:100760008D05E002BA039305E302B803910500008A
:10077000BC039405E402C20399050000C7039F056A
:10078000E702CD03A4050000D203A8050000DB03A7
:10079000AF05EA02E203B405ED02E803B805F00292
:1007A000EE03BD05F302F403C205F602F903C60524
:1007B000F902FE03CA05FC020404CF05FF020B0484
:1007C000D50502030F04D80505031304DB05080350
:1007D0001904E0050B031E04E4050E032704EB05D2
:1007E00011032D04F10514033404F80517033A042A
:1007F000FD051A03410404061D03470409062003EE
:100800004C040E062303520413062603580419064B
:1008100029035E041F062C03660426062F036C04BE
:100820002B063203720430063503770434060000C9
:100830007B04360600007E043906000082043B0675
:1008400000008804400600008E0445060000900465
:100850004706EA0295044B06ED029A044F06F002A1
:100860009E045206F302A3045606F602A8045A0692
:10087000F902AC045D06FC02B1046106FF02B60495
:1008800065060203B80466060503BB046806080390
:10089000C0046C060B03C2046D060E03CA04740682
:1008A0001103CF0478061403D4047C061703D9047B
:1008B00080061A03DE0484061D03E2048706200373
:1008C000E6048A062303E9048C062603EE04900658
:1008D0002903F30495062C03FA049C062F03FF0456
:1008E0009F0632030405A30635030805A606380350
:1008F0000F05AB0600001605B20600001C05B80681
:1009000038032105BC0600002605C00600002B05A3
:10091000C40600009809A4098C097E092E2C3F21E9
:1009200027222D2829402F3A5F3B2B26252A3D3CA4
:100930003E40245B5D5C5E60AAAA2DD4AAAAAA2DC3
:10094000D4AA2DD4AA2DD4AA2DD4AAF0CC335A439C
:100950005100554900333138004A756E2020392046
:10096000323030390031353A35363A3532002047A9
:1009700065727269742044483847484800000D1079
:100980002844002844824428004428100B243E2098
:1009900000322A2400222A140B302838003E281066
:1009A000001028280B3C0A3C003E2A14001C22227E
:1009B00007E08890A09088E007E08890AE9088E0FB
:1009C00007E08884BA8488E007E0868ABE8A86E0E9
:1009D00007E080A8A8A880E007E080A890A880E0B1
:1009E0000503053F0503087F4345494945437F0803
:1009F0001C2214001C223C2046694669534D536555
:100A00007200417573736368616C74656E203F009A
:100A10004E4F43414C4C004E616368726963687489
:100A2000656E0045696E74726167206CF673636869
:100A3000656E3F006D696E004E6F742073656520B2
:100A40006D65004D48204C697374650044657461A0
:100A5000696C7300416273203A2000456D70663AFC
:100A600020005A6569743A004B65696E20456D70C7
:100A700066E46E6765722067657365747A742E200C
:100A8000416E20616C6C652073656E64656E203FFD
:100A900000435100416E736568656E0061757300B7
:100AA00065696E004D736720696E20506F737461C5
:100AB00075732D2067616E672065696E6765726565
:100AC000696874004D657373616765656E747775E9
:100AD00072662061626765737065696368657274C8
:100AE00000454E545755524600537065696368651A
:100AF0007220766F6C6C21204E6963687420676584
:100B000073706569636865727400416C6C65204E32
:100B10006163687269636874656E206CF6736368FC
:100B2000656E203F004B616C747374617274206455
:100B3000757263682D2066FC6872656E3F003C6EBE
:100B40006F63616C6C3E004265657000566962724D
:100B50006100426565702F566962726100204F4BDB
:100B60002000204241434B2000204A612000204EBB
:100B700065696E2000203C2D200020534554200044
:100B8000204D454E55452000204D482000204D5316
:100B90004720003C2D20002D3E20003433342E35DC
:100BA0003030003433392E373030003433342E397E
:100BB000303000EF0B0606F10B3703F80B3812FE4E
:100BC0000B390C040C330B090C32110F0C310200E1
:100BD000000000190C15151B0C2A2A1D0C301B20B7
:100BE0000C2323220C3613280C350A2D0C34140642
:100BF000007071727337DF0074757638FC00777897
:100C0000797A3900646566330061626332E4002EEC
:100C10002C3F2131272D2F3A0015002A00203000CB
:100C200023006D6E6F36F6006A6B6C35006768697D
:100C300034005549007D0C00000000870C31210074
:100C400000980CC4200000590CDB200000A50CC645
:100C500020000000000000000056657273696F6E8E
:100C600000415400425900564552005350454943F3
:100C700048455242454C4547554E4720004552573E
:100C80004549544552540053706569636865726202
:100C9000656C6567756E67004C6976652D6D6F6E66
:100CA00069746F72004E6575737461727400000030
:100CB0000000000000000000000000000000000133
:100CC00002030405060708090A0B0C0D0E0F0002AB
:100CD0000406080A0C0E030107050B090F0D00039B
:100CE00006050C0F0A090B080D0E0704010200048B
:100CF000080C03070B0F06020E0A05010D0900057B
:100D00000A0F07020D080E0B0401090C030600066A
:100D10000C0A0B0D07010503090F0E08020400075A
:100D20000E090F0801060D0A030402050C0B00084A
:100D3000030B060E050D0C040F070A02090100093A
:100D40000108020B030A040D050C060F070E000A2A
:100D5000070D0E0409030F050802010B060C000B1A
:100D6000050E0A010F04070C02090D060803000C0A
:100D70000B0705090E020A06010D0F030408000DFA
:100D80000904010C0805020F0B06030E0A07000EEA
:100D90000F010D03020C09070608040A0B05000FDA
:100DA0000D020906040B010E0C030807050AFF00DB
:100DB00001040208050A030E0907060D0B0C0102C7
:100DC000040803060C0B050A070E0F0D0901F0CCF1
:100DD000335A11241FBECFEFD8E0DEBFCDBF11E0E4
:100DE000A0E0B1E0ECEAF7E502C005900D92A43076
:100DF000B107D9F715E0A4E0B1E001C01D92AC3213
:100E0000B107E1F719D00C94D42BFAC887E187B960
:100E100080E188B984EF8AB98FEF8BB98EE284B90B
:100E200085E085B981E58CBD81E08DBD83E080934F
:100E3000640080936D00089588E10FB6F894809364
:100E40006000109260000FBEE1DF0E94601AFBD1CB
:100E500078940E9430180E9441180E94C41E0E947B
:100E60004F1A0E9476190E9473140E946B190E94F7
:100E7000D3188A9741F48AE09BE060E03DD4882350
:100E800011F00E94A4200E94A51C0E94971E0E949F
:100E900073208AB580618ABD0E94DF100E942219EA
:100EA00064D38091C3029091C4028038910541F4CB
:100EB0000AB403FE03C00E948A1202C00E94E40F1B
:100EC0008091C3029091C4028050904821F489E738
:100ED00091E061E031D58091C3029091C402049702
:100EE000D9F680911D04882319F489E40E94D01951
:100EF00080911D04823019F481E40E94D019809100
:100F00001D04833019F482E40E94D01980911D04DD
:100F1000813019F483E50E94D0190E942219BCCFB8
:100F2000F999FECF92BD81BDF89A80B50895F999DF
:100F3000FECF1FBA92BD81BD60BD0FB6F894FA9A7C
:100F4000F99A0FBE089580914C0190E080FF91E0E6
:100F500080914C018E7F892B80934C0180E0089515
:100F600080914E018F5F837080934E0180E00895E1
:100F700080914F018F5F837080934F0180E00895CF
:100F8000809150018F5F87708093500180E00895B9
:100F900080914D018F5F80934D0180914D01833091
:100FA00010F010924D0180E0089580914C0190E086
:100FB00082FF91E0990F990F80914C018B7F892BD3
:100FC00080934C0180E00895809151018F5F809360
:100FD0005101809151018B3010F01092510180E04D
:100FE000089580914C0190E081FF91E0990F8091EC
:100FF0004C018D7F892B80934C0180E00895809176
:101000004C0190E083FF91E0990F990F990F809127
:101010004C01877F892B80934C0180E008959C01CF
:1010200080914C0183FF05C0C90160EA7AE00C940D
:10103000822AC9016CE97AE00C94822A9C01809191
:101040004C0181FF05C0C90169E67BE00C94822A4E
:10105000C9016EE67BE00C94822A9C0180914C01D0
:1010600082FF05C0C90169E67BE00C94822AC901B0
:101070006EE67BE00C94822A9C0180914C0180FFFB
:1010800005C0C90160EA7AE00C94822AC9016CE9C2
:101090007AE00C94822ABC018091500190E04AE0F1
:1010A00050E00C941D2BBC0180914B0190E04AE074
:1010B00050E00C941D2BBC018091510190E04AE05E
:1010C00050E00E941D2B64E37AE00C94772A9C0187
:1010D00080914D01882321F4C9016BE97BE00FC0A9
:1010E00080914D01813021F4C90163EA7BE007C0A2
:1010F00080914D01823029F4C9016BEA7BE00C94A8
:10110000772A08959C0180914F01882321F4C90119
:101110006CE97AE00FC080914F01813021F4C90160
:1011200067E47BE007C080914F01823029F4C90158
:101130006CE47BE00C94772A80914F01833019F0A6
:1011400080E090E00895C90162E57BE00C94772A85
:101150009C0180914E01882321F4C9016CE97AE059
:101160000FC080914E01813021F4C90167E47BE01A
:1011700007C080914E01823029F4C9016CE47BE004
:101180000C94772A80914E01833019F080E090E032
:101190000895C90162E57BE00C94772A80914B01A8
:1011A0008E5F80934B0180914B01893210F0109239
:1011B0004B010E94761980E0089563E471E048E0F5
:1011C00050E00C94DA2ACF93DF93C8E5D1E08FE0AA
:1011D000FE0111928A95E9F7CE0163E471E048E0DF
:1011E00050E00E94DA2ACE0168E046EB50E020E0B1
:1011F000D4D4882339F083E491E0BE0148E050E084
:101200000E94DA2A80E0DF91CF9108958091520107
:10121000855980936600F999FECF80E090E063E401
:1012200071E040E150E027E937E00E94032B0E9483
:10123000BD14882331F078940E94BD148823E1F70F
:10124000F8940C947314CF93DF93F999FECF83E451
:1012500091E060E070E040E150E020E937E00E947A
:10126000E92AF999FECFC0E1D0E0D2BDC1BDF89A1C
:1012700080B58A3209F43BC081E0809351018BE252
:1012800080934B0180914C01816080934C011092BE
:101290004D0180914C01826080934C0183E08093EA
:1012A000500110924E0110924F0183E491E060E1F1
:1012B0007AE048E050E00E94892AF999FECF80E068
:1012C00090E063E471E040E150E027E937E00E94FC
:1012D000032BF999FECFF999FECF1FBAD2BDC1BD3C
:1012E0008AE280BD0FB6F894FA9AF99A0FBEDF91A0
:1012F000CF9108951F9382E09AE060E0FDD18823AA
:10130000A9F11FB7F8948AB58F7E8ABD8AB58F7D03
:101310008ABD10928B0010928A0010928900109260
:1013200088000E946B1984E20E945E1980E092E8B6
:101330000E9404148BEA8093640084E00E94A41C41
:101340001FBF83B7817F866083BF83B7816083BF00
:10135000889583B78E7F83BF0AB404FEF2CF83E8FB
:10136000809364000E9476190E94731481E01F919B
:10137000089585E39CE061E0DFD280E0089588E68F
:1013800090E060E0D9D242DF80E008950E948A12A6
:1013900080E00895E9ECF2E08AEADF011D928A9587
:1013A000E9F78091DB02887F83608093DB02909174
:1013B0004C01929590728F7D892B8093DB02CF0137
:1013C000449666E947E451E021E0E7D380E00895E0
:1013D000FBD581E0089582E0089586E9EDEDF2E025
:1013E000DF011D928A95E9F781E008958091DB0283
:1013F000887F81608093DB020E94521C882319F051
:1014000084EC9AE002C089EE9AE061E075D181E057
:101410000895CF93DF93C8E5D1E08FE0FE011192EC
:101420008A95E9F7CE0169EC72E00E94BB2ACE01F1
:1014300068E043ED51E020E0B0D3882329F089EC47
:1014400092E0BE010E94BB2A80E0DF91CF91089517
:10145000CF93DF93E9ECF2E001900020E9F73197B8
:10146000E95CF240329708F4D4DFC9ECD2E0FE0127
:1014700001900020E9F73197EC1BFD0B329758F4EF
:1014800088E69AE060E038D1882329F1CE0161E94D
:101490007AE00E94822A8091DB02887F83608093B9
:1014A000DB0290914C01929590728F7D892B8093F5
:1014B000DB020E94521C882319F084EA9AE002C0E1
:1014C00089EE9AE061E018D188E0E9ECF2E0DF0112
:1014D0001D928A95E9F781E0DF91CF91089583E02D
:1014E000089591D080E0089583E29AE060E004D10D
:1014F000811182E00895E9ECF2E088E0DF011D92BD
:101500008A95E9F7CF01449666E940E552E021E08B
:1015100044D381E008950F931F9309EC12E0C801B2
:10152000085F1F4FB80148E050E00E94DA2A045FCC
:101530001F4F86E9F80111928A95E9F7C80166E91B
:1015400046E452E021E029D381E01F910F910895F4
:1015500082E0089581E0089588E7EEE1F4E0DF019C
:101560001D928A95E9F781E008950AB401FE08C04A
:1015700080E060E00E94621980EE99E00E94371AD4
:101580000AB403FE08C087E060E00E94621986EE9C
:1015900099E00C94371A08950F931F93CF93DF931C
:1015A0008C01EB0180E065E00E94621982E06EE749
:1015B0000E944A190115110519F0C8010E94EC1981
:1015C00084E265E00E9462198091C602E82FF0E093
:1015D000EE0FFF1FEC5EF64F859194910E94371A33
:1015E000209761F0CE010E94151A94E5981B892F6F
:1015F00065E00E946219CE010E94EC19DF91CF9143
:101600001F910F910895FF920F931F930E946B19E2
:10161000ACDF89E160E00E94621982E060E80E942C
:101620004A1984E192E00E94EC198DE59BE062E6A4
:101630007BE0B2DF81E060E00E944A1980E061E077
:101640000E94621984E59AE00E94EC1908E511E015
:101650009FE0F92EF8012F2D11922A95E9F7C80184
:1016600061ED72E048E050E00E94DA2AC8010E9471
:10167000F91980E062E00E9462198BE59AE00E940D
:10168000EC19F8012F2D11922A95E9F7C80169ECA0
:1016900072E048E050E00E94DA2AC8010E94F9197D
:1016A00080E063E00E94621982E69AE00E94EC19F1
:1016B000F8011192FA94E9F78091D9029091DA0237
:1016C000B8014AE050E00E941D2B0E94F9190E94C7
:1016D00022198091C3029091C4028050904839F041
:1016E0008091C3029091C4028038910581F781E016
:1016F0001F910F91FF900895FF920F931F938C01FC
:10170000F62E0E946B1980E062E00E94621980E070
:1017100060E00E944A19C8010E94EC19FF2029F0DC
:101720008DE59BE060E070E004C089E69BE06EE63A
:101730007BE032DF0E9422198091C3029091C402A3
:101740008050904811F481E008C08091C3029091CC
:10175000C4028038910571F780E01F910F91FF90CE
:101760000895EF92FF920F931F93CF93DF93962FDD
:10177000682F70E088E2989FC00111240E94602BBE
:1017800022E0E22EE60E00E0FF24C1E0D0E081E599
:101790006F2D0E94621987E08E15A8F0002399F43E
:1017A0008E010E2C02C0000F111F0A94E2F7802F49
:1017B0000E946019802F0E946019802F8A6A0E94FF
:1017C000601901E00BC080E00E94601980E00E9477
:1017D00060198AEA0E94601988EFE80EF39486E0A7
:1017E000F816A9F6DF91CF911F910F91FF90EF901E
:1017F0000895AF92BF92CF92DF92EF92FF920F9334
:101800001F93A090C60283E08093C60210E0BB2421
:1018100003C01BE101C010E00E946B19A6DE8DE53C
:101820009BE062E67BE0B8DEEE24DD2428C0EF2DED
:10183000F0E0E45EF64FC4901F1531F481E06FEFE5
:101840000E944A19BC2C04C081E060E00E944A1941
:10185000802F6E2D0E94621980E20E94D0198C2D7B
:101860000E94D01980E20E94D019F394055F0D34D4
:10187000F1F6E39487E0D80E84E0E81619F0FD2C29
:1018800000E0D5CF0E9422198091C3029091C4023A
:101890000E9469188C3009F4BCCF8D3088F48630F2
:1018A000D9F1873038F4823009F4B5CF833009F0AC
:1018B000B3CF30C08A3081F18B3009F0ADCF10C08A
:1018C0008331A9F0843130F48131F1F0823109F0B3
:1018D000A3CF12C0843131F0853109F09DCF1FC0F4
:1018E00016E09ACF112309F494CF115095CF1B31F4
:1018F00008F091CF1F5F90CF195F1C3108F48CCF97
:1019000017501830E8F788CF173010F41B5E84CFDB
:10191000175082CF15E180CFA092C60203C0A092DB
:10192000C602BB248B2D1F910F91FF90EF90DF908B
:10193000CF90BF90AF9008952F923F924F925F92B9
:101940006F927F928F929F92AF92BF92CF92DF92CF
:10195000EF92FF920F931F93DF93CF9300D000D0AD
:101960000F92CDB7DEB74C016983552436E0252DA3
:101970002F5F239FF0011124E80DF91D85919491AB
:10198000892B11F0522EF3CF44244394BB24B394FB
:10199000F401859194919B838A83252C332493E0D1
:1019A0009093C6020E946B19E0DD89E160E00E941D
:1019B000621982E060E80E944A198A819B810E9434
:1019C000EC19AB2CAA94852D6A2DCBDEA981AA2314
:1019D00009F039C08AE79BE062E67BE0DDDD80E06C
:1019E00060E00E944A1980E062E00E946219B6E05D
:1019F000BB9E80011124080D191DF8018591949159
:101A00000E94EC19F8013496059114910115110505
:101A100009F464C081E060E00E944A191092580104
:101A200088E591E0F801099588E591E00E94271A80
:101A3000E1E5E81B8E2F63E00E94621988E591E0E2
:101A40000E94F9194BC0F981F13009F047C08DE5CA
:101A50009BE062E67BE0A0DD6B2C7724842D90E098
:101A60000396861597051CF45DEF452E4B0CB414B8
:101A700008F44B2CC42CDD24C601880F991F8C0D53
:101A80009D1D880F991F880D991D9D838C8300E0F3
:101A900010E07801EC0CFD1C2E143F04FCF0602FCC
:101AA0006F5F80E00E946219E614F70419F481E088
:101AB0006EEF02C081E060E00E944A19EC81FD8176
:101AC000859194910E94EC190F5F1F4FAC81BD81ED
:101AD0001696BD83AC8304301105D9F60E942219F5
:101AE0008091C3029091C4028050944011F0AB2CBD
:101AF00004C0E1E0EB1508F0A52C8091C3029091A1
:101B0000C4028050904211F0BA2C07C0A51418F0FE
:101B1000BB24B39402C0BA2CB3948091C3029091B9
:101B2000C4028038910511F480E01FC08091C30287
:101B30009091C402049741F08091C3029091C40235
:101B40008050904809F02BCF86E0B89EF001112418
:101B5000E80DF91D329685919491009709F41FCFF5
:101B6000FC010995882309F41ACF0F900F900F906C
:101B70000F900F90CF91DF911F910F91FF90EF90F9
:101B8000DF90CF90BF90AF909F908F907F906F909D
:101B90005F904F903F902F9008952F923F924F92D9
:101BA0005F926F927F928F929F92AF92BF92CF92ED
:101BB000DF92EF92FF920F931F93DF93CF93CDB7F6
:101BC000DEB728970FB6F894DEBF0FBECDBF6C010D
:101BD000462E1A01298381E08093C602FF249924AE
:101BE0005524262F30E03B832A83215030403D830B
:101BF0002C830E946B19B9DCF60101900020E9F7F3
:101C000031978E2E8C182114310489F082E060E81F
:101C10000E944A19C1010E94151A86953AE2381BA2
:101C2000832F60E00E946219C1010E94EC1982E0DA
:101C300060E00E944A1982E460E00E946219682C08
:101C400077248A819B818619970963E571E04AE0D0
:101C500050E00E941D2B0E94F919FF2019F065E742
:101C60007BE002C062E67BE08981882319F080E88E
:101C70009BE002C08DE59BE08FDC81E060E00E948C
:101C80004A1990E010E000E0EE2411C0EC0DFD1DBB
:101C900080819E830E94041A180F9E81123528F4B9
:101CA000F91609F4E02E9F5F02C00F5F10E0E92FE4
:101CB000F0E06E167F0654F7802F6E2D52DDF9147A
:101CC000A0F410E010C0F601E90DF11D80810E9422
:101CD000041A282F812F90E0820F911D82359105E3
:101CE00024F4120F9A94992071F75F1438F5192D86
:101CF000EE240EC01815F9F0F601E10FF11D8081F8
:101D00000E94041A080F023510F41F5F02C0E3940A
:101D100000E01F1578F30FC010E0981451F0F601A1
:101D2000E90DF11D939480810E94041A180F123559
:101D3000A0F39A94EA9493E09E1570F3592CEE2444
:101D4000BB24AA24B39480E06B2D0E94621900E0AA
:101D500010E01FC05F1441F4EE2031F48FEF0E94B9
:101D60006019A12EEE24E394EF81F88580810E9412
:101D7000041A282F802F90E0820F911D8235910543
:101D80008CF4020FEF81F88580810E94D019539462
:101D90001F5F9601250D311D38872F83F901808142
:101DA0008823C1F6EE2039F4581429F48FEF0E94ED
:101DB0006019EE24E394F4E0BF1621F60E94221984
:101DC0008091C3029091C402892B09F412CF8091B3
:101DD000C3029091C4020E946918282F833109F42C
:101DE00097C0843148F48131E9F1823108F059C05B
:101DF000863009F0A7C01BC0853149F0853108F451
:101E000082C0833219F18A3209F09CC08DC0FF2054
:101E100009F4BCC0FA948F2D90E0BC016F5F7F4F36
:101E20006C0D7D1D8C0D9D1D0E94BB2AE2CE29816B
:101E3000222309F4ADC089EA91E061E07DDD8130C3
:101E400009F4C0C0823008F4D4CEA2C08091C6028A
:101E50008F5F0AB400FE02C0837001C0817080935E
:101E6000C602C7CEEF2CEA1809F4C3CE1E2D00E03F
:101E7000F601E10FF11D80810E94041A080F02355E
:101E800010F41150A9F78A2D90E0AC01410F511DBB
:101E90002F2D30E0281B390B421753078CF1FE2CF5
:101EA000A8CE1F2D1A1900E00DC0F601E10FF11D9B
:101EB00080810E94041A080F023518F0F12E00E00C
:101EC00004C01F5F181588F3F9CFF81451F0F6011C
:101ED000EF0DF11DF39480810E94041A080F023562
:101EE000A0F32A2D30E0210F311D2615370514F0FF
:101EF000F82C7FCE8F2D90E0281739070CF079CE83
:101F0000F12EFA0C76CEFF2009F473CEFA9471CE3E
:101F10008F2D90E0EC81FD818E179F070CF069CE2C
:101F2000F81408F066CE30C00AB400FC06C08091F8
:101F3000C202882311F020E002C05BDC282F8AB5A2
:101F40008E7F8ABD203208F454CEF41419F00AB4FE
:101F500000FE04C08AB581608ABDFA940AB400FC10
:101F60000FC0942D07C0F601E90FF11D8291319643
:101F700080839150F916B8F3F601E80DF11D118236
:101F8000F601EF0DF11D2083F39433CE80E001C004
:101F900081E028960FB6F894DEBF0FBECDBFCF917B
:101FA000DF911F910F91FF90EF90DF90CF90BF9046
:101FB000AF909F908F907F906F905F904F903F90E9
:101FC0002F900895FF2415CE2F923F924F925F924B
:101FD0006F927F928F929F92AF92BF92CF92DF9239
:101FE000EF92FF920F931F93CF93DF9383E0809341
:101FF000C60299249394FF24F39498E5292E91E046
:10200000392E8DED482E82E0582E06E9802E0E9452
:102010006B19ABDA89E160E00E94621982E060E846
:102020000E944A1983E49AE00E94EC19EF2CEA948A
:102030008AE06E2D96DB80E89BE062E67BE0ACDA1E
:10204000AF2CBB24892D90E003968A159B051CF4C8
:102050001DEF912E9F0CF91408F49F2C00E010E066
:10206000C92CDD243601089461087108E801CC0D03
:10207000DD1DCB30D105ECF5602F6F5F80E00E9455
:102080006219CA15DB0539F482E06EEF0E944A1925
:1020900081E06EEF06C082E060E00E944A1981E0B4
:1020A00060E00E944A19F1012FE011922A95E9F7A8
:1020B000C301800F911FBC01660F771F680F791F46
:1020C000660F771F660F771F6E5D7B4F88E591E087
:1020D00048E050E00E94DA2A80E20E94D01988E5A8
:1020E00091E00E94F9190F5F1F4F0430110509F0AC
:1020F000BDCF0E9422198091C3029091C4028050EA
:10210000944019F4F1E0FF1508F0EF2C8091C30220
:102110009091C4028050904231F489E08E1518F0FD
:10212000FE2CF39401C0FE2C8091C3029091C40256
:1021300080389105A1F481E0DF91CF911F910F913B
:10214000FF90EF90DF90CF90BF90AF909F908F90D7
:102150007F906F905F904F903F902F900895809167
:10216000C3029091C4028050904809F050CF84E897
:1021700092E061E0E1DB823009F049CF8F2D90E001
:102180000197BC01660F771F680F791F660F771FD5
:10219000660F771F6E5D7B4F89EC92E048E050E060
:1021A0000E94DA2AF201282D11922A95E9F78DED85
:1021B00092E066E94DE752E021E0EFDC28CF0F9393
:1021C0001F93CF93DF930E946B19CFD981E460E016
:1021D0000E94621982E060E00E944A1920919604F0
:1021E0003091970484E690E0AC01249FC001259FC4
:1021F000900D349F900D112460E770E00E944C2BED
:10220000CB01C8E5D1E0BE014AE050E00E941D2BA1
:10221000FE0101900020E9F7EB55F14041F480E325
:102220000E94D0198EE20E94D019CE0109C080917F
:1022300058010E94D0198EE20E94D019CE01019659
:102240000E94F91986E50E94D01983E08093C602A6
:102250000AB403FE05C080E89BE06DE87BE004C0A3
:1022600080E89BE068E87BE097D988E160E00E9425
:10227000621982E060E00E944A1988EF99E00E94AA
:10228000EC1980E060E00E944A1908E511E08FE057
:10229000F80111928A95E9F7C80163E471E048E01A
:1022A00050E00E94DA2AC8010E94271A982F9695BA
:1022B0008AE2891B62E00E946219C8010E94F91932
:1022C000DF91CF911F910F9108953F924F925F92AE
:1022D0006F927F928F929F92AF92BF92CF92DF9236
:1022E000EF92FF920F931F93CF93DF93EC01462E53
:1022F00081E08093C6025B8858E0652E712C6C0EDD
:102300007D1EA62EBB2445E0AA0CBB1C4A95E1F716
:1023100032E1832E912C8A0C9B1CCC242AE2322E93
:102320008A89877090E08430910534F48230910579
:1023300084F4019729F506C086309105A4F006972C
:10234000F9F407C088E591E061EE7AE00E94822A04
:1023500017C088E591E067E97BE00E94822A8BE55F
:1023600091E0BE0109C088E591E063E97BE00E944D
:10237000822A8BE591E0B30148E050E00E94DA2A1E
:10238000AAD7F3D880E89BE062E67BE005D982E03B
:1023900060E880D788E591E00E94271A8695232D72
:1023A000281B822F60E08ED788E591E00E94F91902
:1023B00081E060E06FD7DC2CEE24E39480E06E2DAA
:1023C00081D7FF2414C08E010D0D111DF8018489E1
:1023D0000E94041A282F8F2D90E0820F911D8235C4
:1023E00091053CF4F20EF8018489DAD7D394D51420
:1023F00050F3F4E0EF1609F725D78091C3029091CE
:10240000C402892B71F08A898770853051F48AB5AE
:10241000877F8ABD6A89687F64606A8BC4010E9475
:10242000301F8091C3029091C40224E08030920753
:1024300009F441C0E4E081309E0728F4803891051A
:1024400009F06ECF55C0F0E280309F0729F0805030
:10245000904809F065CF02C010E047C08CE192E0DF
:1024600061E06ADA823021F4842D0E940C2040C0A1
:102470008330E9F46A89862F8770863019F08230BC
:10248000B9F506C0687F6360C4010E94301F48CF61
:102490000E94C51C998B888B8A89887F83608A8B70
:1024A000C501BE0144E150E00E944A1F21C08823BB
:1024B00009F436CF1DC0CC2009F432CF10E0FE0164
:1024C000EC0DF11D8489A0D7180F123508F028CF24
:1024D000CA94A9F725CFFE01EC0DF11D848994D78C
:1024E000180F123508F01CCFC394C514A0F318CFF1
:1024F000DF91CF911F910F91FF90EF90DF90CF90E0
:10250000BF90AF909F908F907F906F905F904F9013
:102510003F9008952F923F924F925F926F927F92D9
:102520008F929F92AF92BF92CF92DF92EF92FF92E3
:102530000F931F93DF93CF93CDB7DEB72A970FB6D4
:10254000F894DEBF0FBECDBF33243394DD24D39483
:1025500001C0D62C21E130E07724F999FECF32BDBD
:1025600021BDF89A80B5811173942F5F3F4F81E0B0
:102570002131380791F7772019F48AB5877F8ABD12
:1025800093E09093C602A7D60E94B50A89E160E065
:1025900099D682E060E87ED687E19AE01DD76D2C5F
:1025A0006A94872D662DDDD884E99AE062E67BE0A7
:1025B0000E94CC0AED2DF0E0FC83EB83832D90E0AC
:1025C00003968E179F071CF45DEF352E3D0CD31438
:1025D00008F43D2C222400E010E0232D30E03E835F
:1025E0002D83872D90E098878F83ED80FE80E00E0D
:1025F000F11EEF81F885EE15FF050CF4A2C0602FE7
:102600006F5F80E05FD630E0CC242FEF0DC0F999EA
:10261000FECF822F90E08F5E9F4F92BD81BDF89AD2
:10262000C0B4C1103F5F2150832F90E08E159F05ED
:1026300074F32C2D30E045E0220F331F4A95E1F76B
:102640003A872987C90169EC72E04EE150E00E94A7
:10265000791F89EC92E061E97AE00E94642A2C01FA
:102660008091DB02877090E08330910501F1843026
:10267000910534F48130910561F0029799F512C00B
:1026800085309105F1F085309105B4F0069751F54C
:1026900021C020ED822E29E0922E9DEDA92E92E000
:1026A000B92E20C088EC882E89E0982E17C0B0EC97
:1026B0008B2EB9E09B2E12C0A0EB8A2EA9E09A2E99
:1026C00004C0F8EB8F2EF9E09F2EE1EDAE2EE2E094
:1026D000BE2E08C078ED872E79E0972E69ECA62EE5
:1026E00062E0B62EC401C3D681E060E0D3D580E2BB
:1026F00057D68B819C81E816F90641F481E06EEF94
:10270000C9D5E985FA85FA83E9832C2CE8E5F1E05F
:102710002FE011922A95E9F788E591E0B50148E0AC
:1027200050E00E94DA2A452819F48FEE99E09FD6EE
:1027300088E591E05ED60F5F1F4F0430110509F068
:1027400054CF80D58091C3029091C40280509440B0
:1027500019F481E08D1508F06D2C8091C3029091E1
:10276000C4028050904219F4671408F46394809175
:10277000C3029091C40280389105D1F480E02A967A
:102780000FB6F894DEBF0FBECDBFCF91DF911F9182
:102790000F91FF90EF90DF90CF90BF90AF909F9000
:1027A0008F907F906F905F904F903F902F90089503
:1027B0008091C3029091C402049741F08091C302BA
:1027C0009091C4028050904809F0C3CE222009F4B1
:1027D000C0CE89819A8169EC72E044E150E00E94A8
:1027E000791F4091DC0250E04B5E5F4F89819A81F6
:1027F00069EC72E00E94791F23E02093C60289EC05
:1028000092E0622D62DDA5CE4FB7F8949C015D98F1
:102810003EBD0DB407FEFDCF8EB5382F2EBD0DB4D5
:1028200007FEFDCF8EB5282F5D9A4FBFC9010895D1
:10283000906AEACF80E090E0E7CF88EC92E8E4DFAE
:1028400080ED97E00197F1F781E89AECDDDF83E80E
:102850009AECDADFEFDF80E090EBD6DF409841982A
:10286000429A8AB58D7F8ABD10920401089582E054
:10287000809304018091960490919704823E910583
:1028800020F040984298419A03C040984198429A5B
:1028900088E092E8B9DF88E392E8B6DF8AB5826023
:1028A0008ABD08959B01AC01283185E1380780E09D
:1028B000480780E0580760F460E678EA80E090E03E
:1028C0000E94732BDA01C90101978068966C0AC0D7
:1028D0006CEF72E485E090E00E94732BDA01C9018D
:1028E0000197966C91CF88EE93E028EC30E0F901E7
:1028F0003197F1F70197D9F780EE90EC85DF87EDFE
:1029000090E882DF8CEA92EC7FDF81E89AEC7CDF52
:1029100080E090EE79DF80E098EC76DF87EF94EC52
:1029200073DF8BDF80E197E20197F1F788E097E0B2
:102930007FDF80914D01813019F488E29FE078DFDC
:1029400080914D01823019F487EA97E071DF88EABF
:1029500094E95ADF60E875E280E090E0A3DF80E46C
:1029600098E952DF6ADF66DF8AB18AB95B9A88E04C
:102970008093690082E08DBB0895809104018111EC
:1029800081E008951F920F920FB60F9211240F93BA
:102990001F932F933F934F935F936F937F938F93E7
:1029A0009F93AF93BF93EF93FF9344DF97FF2AC0AA
:1029B00080910401813041F0813018F0823011F5AE
:1029C0001DC081E08093040181E8BED780E090EBD8
:1029D0001BDF8C0181E0A6D7802F27D0882319F038
:1029E0002CDF1092040180910501823058F0809113
:1029F0003501882339F481E0A7D704C0E7D190E0FE
:102A0000986B02DFFF91EF91BF91AF919F918F91F2
:102A10007F916F915F914F913F912F911F910F91F6
:102A20000F900FBE0F901F901895CF92DF92FF92DC
:102A30000F931F93CF93DF93F82EC0900801D0908F
:102A4000090180910B01C82FD0E080913501082F3A
:102A500010E080910501823009F467C0833030F4C2
:102A6000882371F0813009F08FC144C0843009F4AB
:102A70001AC1843008F4CBC0853009F085C182C109
:102A8000FE01E859FE4FF0822196CE0104978B306B
:102A90009105B8F488599E4F0E94242A882389F40E
:102AA00080914C0183FF09C081E08093050184E09F
:102AB0008093C70200E010E080C18FEF8093050192
:102AC0007CC1C130D10519F4CC24CA94DC2CC601D8
:102AD0006F2D0E944C2A6C01C431D10509F05CC1F4
:102AE00082E08093C70280917B018A5E80930A0115
:102AF00083E044C1F801E854FB4FF0820F5F1F4FA1
:102B00000331110509F048C182E08093050110925C
:102B1000360110923701109239011092380180E08D
:102B2000C0E0D0E00FE010E038C1FE01E859FE4FF0
:102B3000F0822196C130D10519F4CC24CA94DC2C42
:102B4000C6016F2D0E944C2A6C01C431D10531F4AD
:102B500083E0809305018CEA80930A01CE018370A3
:102B60009070892B09F018C178948091360160919A
:102B7000370190E070E068547B4F88599E4F40E0E9
:102B800028E00E940C29282F843030F08FEF8093AA
:102B9000050188EC90E02BC0809136018C5F80931A
:102BA0003601809137018D5F809337018091380124
:102BB00090913901820F911D9093390180933801D2
:102BC000C431D10508F4E8C080917B018823A1F0CD
:102BD00080917B018A5E80930A0180917B01873915
:102BE00008F4DAC08FEF8093050180EF90E09093B6
:102BF00039018093380137C08FEF8093050187E951
:102C000090E09093390180933801AED1C5C0FE01A8
:102C1000E859FE4FF0822196C6016F2D0E944C2A82
:102C20006C0120910A01822F90E0C817D90709F0A2
:102C3000B3C0273120F0FE01EA59FE4F1082011582
:102C4000110599F486E990E0909339018093380159
:102C5000C114D10429F485E080930501789484D1CE
:102C60008FEF8093050181E098C084E08093050197
:102C700080917B0190E0880F991F69E070E00E94CD
:102C8000602B6F5F7F4F8B01000F111F060F171F07
:102C9000265120930A0110923701109236011092AA
:102CA0003A0180E03CC080913701E82FF0E0E85421
:102CB000FB4FF0828F5F809337012196C330D1059F
:102CC00009F04EC08091370190E08017910711F014
:102CD00029E009C08091360190913A0120910A01C2
:102CE000281B220F291B78948091360160913701AF
:102CF00040913A0190E070E06B547B4F84589E4FB6
:102D00000E940C29282F843068F08FEF80930501F2
:102D100089EC90E0909339018093380181E0C0E024
:102D2000D0E03BC0809136018C5F8093360190915A
:102D3000360180913A01890F8093360180913801E4
:102D400090913901820F911D909339018093380140
:102D500080913A0191E0892780933A01C0E0D0E068
:102D60008091370190E080179107B4F080EA90E0FD
:102D70009093390180933801F7D08FEF809305014C
:102D800080E007C0000008C01092050181E0C0E0AB
:102D9000D0E000E010E001C080E0D0920901C092D4
:102DA000080100933501C0930B01DF91CF911F9172
:102DB0000F91FF90DF90CF900895C0E0D0E087CED4
:102DC0003CDD85E08093670181E0BEC590912702DC
:102DD00080910601833009F45AC0843030F4813088
:102DE000B1F1823008F041C00AC0853009F46FC0EB
:102DF000853008F456C0863009F095C07EC08091B9
:102E00004C01E091070183FF14C0E33160F484E0DA
:102E10008093C702EF5FE0930701E150F0E0E45CCC
:102E2000F64F849108951092070181E08093060186
:102E30000EC082E0809306018093C702EF5FE093AB
:102E40000701E150F0E0E85CF64F8491089520918D
:102E500007012F3028F4E22FF0E0E854FB4F2DC09B
:102E60001092070182E080930601E0910701E430AF
:102E700048F4EF5FE0930701E150F0E0E85CF64FC3
:102E8000849108951092070183E0809306012091B8
:102E90000701243118F4E22FF0E00DC084E08093A4
:102EA000060120910701E22FF0E0892F90E044967F
:102EB000E817F90738F4EC5EFD4F80812F5F20930F
:102EC0000701089585E08093060110920701909113
:102ED0000701923028F4E92FF0E0E254FD4F17C0CB
:102EE0001092070180914C0183FD04C087E080931C
:102EF000060117C086E0809306019091070180913A
:102F00003501981748F4E92FF0E0E953FB4F808131
:102F10009F5F90930701089587E0809306011092C8
:102F200035018AEA0895109207011092060148DFE0
:102F30008AB58D7F8ABD80E008951FDD882329F042
:102F400078941BDD8823E9F7F894109206018FCC62
:102F500014DD882319F081E090E008956BDC892F5F
:102F60009927817090700895CF93DF9388E691E060
:102F700062E579E00E94642AEC0180914C0182FDB7
:102F800002C020E00AC088E691E06FE479E00E9488
:102F9000642A20E0892B09F421E0CD2B51F0222373
:102FA00041F488E691E063E471E00E94A82A892B4D
:102FB00081F440917B0150E04B5E5F4F83E793E0EB
:102FC00068E671E00E94982A8AB580688ABD81E02F
:102FD00000C0DF91CF910895EF92FF920F931F935E
:102FE000CF93DF937C0180E09DD40FEF1FEFC0E013
:102FF000D0E009C0FE01EC5EFD4FC80160810E9477
:103000004C2A8C012196F701838990E04496C817D9
:10301000D90780F380914C0183FF05C0C70168EB9D
:1030200074E00E9487241093BF020093BE0285DFE4
:1030300080914C0183FF0AC0C701449667EC74E09D
:10304000F70143890E94EF218093350180E07CD411
:1030500080E0DF91CF911F910F91FF90EF90089545
:1030600082E08093C6021092C4021092C3021092B2
:10307000C1021092C002E8E6F0E0808184608083A3
:1030800008959FB7F894E8E6F0E08081846080833B
:10309000509A519A58985998589A599A50988AB172
:1030A0008C7F8AB99FBF08951F920F920FB60F921F
:1030B00011248F93EF93FF93E8E6F0E080818B7FFC
:1030C0008083FF91EF918F910F900FBE0F901F9013
:1030D00018959C018AB58E7F8ABD4FB7F8948FE111
:1030E0008093C2028091C0029091C102821793071F
:1030F00049F48091C5028F5F8093C5028AB58160D3
:103100008ABD02C01092C5023093C1022093C00252
:103110004FBFEFE0E15021F03695279520FFFACF21
:103120008091C602833059F41092C502F0E0EE0F90
:10313000FF1FEE0FFF1FEA54F44F84910895F0E053
:10314000823051F41092C502EE0FFF1FEE0FFF1FE9
:10315000EB54F44F849108959FB7F894EE0FFF1F3E
:10316000EE0FFF1FED54F44F2591349121153105D9
:1031700019F49FBF80E008958091C502F901E80F1E
:10318000F11DE491EE2331F480E0F8CF8E2F90E032
:103190000C94952B8093C5029FBF8091C60281300D
:1031A000A9F38E2F08951F9319B11370133019F4DA
:1031B00080E090E03DC084E0B5D380914C0180FF79
:1031C00006C00AB404FE03C08AB580628ABD20E04E
:1031D00030E0412F10FF0CC05C985098519A0000CD
:1031E0005C9A1EBC0DB407FEFDCF51988EB5282FFA
:1031F00041FF0CC05C98509A519800005C9A1EBC2C
:103200000DB407FEFDCF50988EB5382F1092680090
:1032100083E08BBB309342012093410184E094D33F
:10322000809141019091420110924201109241011E
:103230001F910895B8DF009721F09093C402809306
:10324000C3020895CF93DF93C0E2DEE410C00BB455
:1032500000FE0AC01092C4021092C3028BB58E7F8A
:10326000EAE4F0E0818313C0CE010197F1F79BDF20
:10327000892B69F307C00BB400FC09C0CE0101978C
:10328000F1F702C0C0E2DEE4D5DF892BA1F7DF91C0
:10329000CF91089580930C0160930D0108952FB78D
:1032A000F8949FEE9BB98EBD5A9861115A9A0DB44D
:1032B00007FEFDCF8EB55C9A2FBF089560E0EFCF7B
:1032C00061E0EDCF1F93162F8058F8DF812F805CCF
:1032D000F5DF1F910895CF93DF93C8EFD1E080E031
:1032E000EFDF2197E1F7DF91CF91089510920D0163
:1032F00081E080930C01449880ED97E0FC013197C8
:10330000F1F7449A0197F1F780E29EE40197F1F713
:1033100081E2D4DF80914B01885D8068CFDF86E059
:10332000CDDF83E1CBDF80E2C9DF8CE0C7DFD3CF25
:10333000982F8B3718F18F3DD1F0803E38F4863DC1
:1033400069F18C3D61F0843CA1F407C0863F59F0DF
:103350008C3F59F0843E69F404C09BE70FC09DE7A1
:103360000DC09EE70BC09FE709C090E807C091E839
:1033700005C0923818F080E090E00895905283E004
:10338000989FF001112480910C01E80FF11DEE0FC0
:10339000FF1FE853F94F8591949108959CE7EECF74
:1033A0000F931F93CF93DF93C3DFEC01009761F07E
:1033B0008E012196F8010491802F8E7F90910D014E
:1033C00089277EDF00FFF4CF80910D0179DFDF9147
:1033D000CF911F910F910895CF93DF93EC0101C01E
:1033E000DFDFFE01219684918823D1F7DF91CF9111
:1033F0000895CF93DF93EC0101C0D2DF8991882338
:10340000E1F7DF91CF91089593DF009711F440E049
:1034100009C09C01F9012F5F3F4FE491422F481BE7
:10342000E0FFF8CF842F8F5F08951F93CF93DF9332
:10343000EC0110E002C0E8DF180FFE012196849134
:103440008823C9F7812FDF91CF911F9108951F9392
:10345000CF93DF93EC0110E002C0D6DF180F899103
:103460008823D9F7812FDF91CF911F910895FF9283
:103470000F931F93CF93DF93EC018C01FC01F49029
:1034800004C02196FE0184911BDF9E01201B2F1595
:10349000C0F3DF91CF911F910F91FF90089510928B
:1034A000C70282EA8093800081E0809381001092BD
:1034B00089001092880010928B0010928A00089563
:1034C000109216011092180110921D04109217010B
:1034D0000895FF920F931F93CF93DF938BB58D7F4A
:1034E0008BBD90E8F92E01E0F999FECFF999FECF56
:1034F000802F90E08F5E9F4F92BD81BDF89A80B57E
:10350000882319F1C82FD0E085E0CC0FDD1F8A9504
:10351000E1F7CE0169E171E044E150E0EAD41091B5
:103520002B01812F8770863081F489E191E06EE074
:1035300071E048E050E00E94C22A892B31F4187FE4
:103540001360CE014296612F8BD4FA940E5FFF2058
:1035500059F6DF91CF911F910F91FF9008950F932E
:103560001F93CF93DF930AB407FEE7C080918503D2
:10357000869586958695837090E08130910509F453
:1035800043C083309105A9F0892B09F0C3C08BE7B4
:1035900093E043D30BB401FCBDC08EE091E06BE738
:1035A00073E048E050E00E94DA2A8BB582608BBD60
:1035B000B1C0209124023091250280918303909123
:1035C00084032817390709F0A5C084E192E06BE76E
:1035D00073E048E050E00E94C22A892B09F09AC0AB
:1035E0000091160110E045E0000F111F4A95E1F728
:1035F0000E5E1F4FC80115D4682F687F6260C80136
:103600002FD410921D0486C001E110E0F999FECF7D
:1036100012BD01BDF89A80B5882329F1C82FD0E0EA
:1036200035E0CC0FDD1F3A95E1F7CE014296F9D394
:103630008C5F87708230B8F4CE0169E171E044E1BB
:1036400050E057D420918303309184038091290165
:1036500090912A012817390731F4909186038091BF
:103660002C01981769F10F5F1F4F81E00131180796
:1036700069F654C0802F90E0412F50E025E0880F7C
:10368000991F2A95E1F763E773E004D4802F612F37
:10369000FDD48AB580628ABD8AB588608ABD8BB543
:1036A00081608BBD80914E0180FF03C080E28093DA
:1036B000C70280914E0181FF03C088E08093C80259
:1036C00083E793E061E97AE00E94642A892B11F193
:1036D0008CE192E063E471E048E050E00E94DA2A75
:1036E00084E192E06BE773E048E050E00E94DA2A60
:1036F0001092270280912602886180932602809191
:10370000780190917901909325028093240282E0C0
:1037100080931D048AB58F778ABD0FC08091850381
:10372000887F85608093850310917B011B5E812FCC
:1037300047D4082F882371F39DCFDF91CF911F913C
:103740000F9108950F931F93CF93DF9316D988237A
:1037500009F0A3C080911D04813009F472C081304A
:1037600038F0823009F48FC0833009F096C03EC033
:103770001FEFF999FECF809118018F5F8093180198
:10378000F999FECF90E08F5E9F4F92BD81BDF89A70
:1037900000B5002331F1C02FD0E075E0CC0FDD1F64
:1037A0007A95E1F7CE0142963CD387708330C9F415
:1037B00084E08093C702CE0164E172E04AEA50E0FF
:1037C00098D3009316018091500190E063E0880F38
:1037D000991F6A95E1F78093170181E080931D049A
:1037E0005CC0112309F459C01150C3CF10921D04BD
:1037F00084E192E060E070E04AEA50E00E94A12A91
:103800008CE192E063E471E048E050E00E94DA2A43
:1038100084E192E062E37CE048E050E00E94892A83
:1038200080912602877E8093260280912602887FDF
:103830008360809326021092270284E08093C7025F
:1038400029C080911701882351F08150809317017E
:103850008F5F90E087709070892BF9F41BC0009106
:10386000160110E055E0000F111F5A95E1F70E5EAA
:103870001F4FC801D6D2682F687F6660C801F0D29A
:1038800010921D040AC08091180181508093180184
:1038900010921D0484E192E09FDBDF91CF911F9194
:1038A0000F910895FF920F931F938091DB02877E03
:1038B00088608093DB0281ED92E063E471E048E090
:1038C00050E00E94DA2AEDEDF2E001900020E9F7E5
:1038D000EE5DF240E093DC0258D09093DA028093E0
:1038E000D9020091DC020B5EFFB6F894802F68D3FA
:1038F000182F882319F4FFBE80E010C090E0402FFD
:1039000050E0E5E0880F991FEA95E1F769EC72E075
:10391000C1D2812F602FBAD3FFBE81E01F910F91DA
:10392000FF90089590912E01982B90932E019FB7B0
:10393000F894E1E6F0E080E88083108287E08093ED
:10394000B1001DBC9FBF089508958EE180933101A1
:1039500023E0209330018091510190E09093340155
:103960008093330116BC10926E0025BD1092850025
:1039700010928400109232018FE180932F011092F7
:10398000B20081E080937000089580913D01909194
:103990003E01A0913F01B091400108951F920F9206
:1039A0000FB60F9211242F933F934F935F936F9312
:1039B0007F938F939F93AF93BF93EF93FF9382E097
:1039C000B1DF8091C202882329F41092C1021092C3
:1039D000C00205C08091C20281508093C2020AB425
:1039E00004FE78C040912F0140FF20C02091C70203
:1039F0002223E1F084E59CE6A4E1BDEA022E04C0A6
:103A0000B695A795979587950A94D2F780FF07C03A
:103A100088ED90E0909389008093880004C0109214
:103A200089001092880021502093C7020AB405FE35
:103A300017C080918A0090918B00809621E0803E93
:103A4000920738F490938B0080938A001092320191
:103A50001CC08FEF91E090938B0080938A0015C07B
:103A600020918A0030918B0080918A0090918B0088
:103A7000409738F02051304030938B0020938A00DB
:103A800004C010928B0010928A000AB401FC18C086
:103A90004F3011F04423A1F42091C802222381F079
:103AA00088EA90E0022E02C0959587950A94E2F785
:103AB00080FF02C0409A01C0409821502093C80264
:103AC00080913201815080933201882319F48AB5A4
:103AD0008F7D8ABD80912D01882309F08DC0809152
:103AE0003501882309F088C081E080932D01789406
:103AF00036DD80912F018F3009F424DE30912F01C3
:103B0000343111F580915101882309F470C08091FE
:103B1000330190913401009789F480911D0488232A
:103B200009F065C083E08093C70280931D048091F3
:103B300051012CE3829FC001112401C00197909391
:103B400034018093330153C0332309F050C0809176
:103B50003D0190913E01A0913F01B091400101963D
:103B6000A11DB11D80933D0190933E01A0933F01A3
:103B7000B09340018FE180932F010AB404FC1AC076
:103B8000499905C0809168008460809368000BDBD0
:103B90008038910521F480913001815001C083E08B
:103BA0008093300180913001882321F58AB58061AE
:103BB0008ABD20C0F8DA8034910521F4809130016B
:103BC000815001C083E080933001809130018823CF
:103BD00009F4000080913101882329F48EE180935B
:103BE0003101D2D007C081508093310103C03150E0
:103BF00030932F0110922D01FF91EF91BF91AF9162
:103C00009F918F917F916F915F914F913F912F91F4
:103C10000F900FBE0F901F901895CF92DF92FF92DA
:103C20000F931F93CF93DF936C0100E010E0F02E11
:103C3000E801CC0FDD1FC00FD11FCC0FDD1FCC0F53
:103C4000DD1FBE016E5D7B4FC60148E050E00E9463
:103C5000C22A892B59F4FE01E25EFB4F208131819B
:103C6000428153818AE0081741F41AC00F5F1F4F49
:103C70000A301105E1F62AE014C080913D019091CF
:103C80003E01A0913F01B0914001821B930BA40B18
:103C9000B50B89559240A040B04010F4202F25C0AC
:103CA0002F2D8AB580628ABD80914F0180FF03C0AD
:103CB00084E08093C70280914F0181FF16C086E0A7
:103CC0008093C80212C02A3070F4239FC0011124CF
:103CD000DC01A25EBB4FFC01EE5EFB4F8CE001906D
:103CE0000D928150E1F7215001C03CE0222359F7A9
:103CF00082E294E0B60148E050E00E94DA2A809126
:103D00003D0190913E01A0913F01B091400180930F
:103D10001E0490931F04A0932004B0932104DF910C
:103D2000CF911F910F91FF90DF90CF9008950F9347
:103D30001F93CF93DF93EEE1F4E088E7DF011D925C
:103D40008A95E9F78F01C0E0D0E0F8011082118276
:103D500012821382CE01880F991F8C0F9D1F880F2E
:103D6000991F880F991F8E5D9B4F60E17AE00E943A
:103D7000822A2196045F1F4FCA30D10531F7DF91A7
:103D8000CF911F910F91089580E880BF3D9AE4E69E
:103D9000F0E080818E7F80831092970410929604C9
:103DA00087E480937C008DED80937A0008951F92C4
:103DB0000F920FB60F9211248F939F933D9880918D
:103DC0007800909179008135910540F080917800DC
:103DD00090917900909397048093960480917A0053
:103DE0008F7780937A008091640081608093640073
:103DF0009F918F910F900FBE0F901F9018958EBDC1
:103E00000DB407FEFDCF08955F9885E0F8DF80E0F0
:103E1000F6DF5F9A0EB400FCF7CF82E08A95F1F7E7
:103E20000895FF920F931F938C01FFB6F894ECDF77
:103E30005F9883E0E4DF812FE2DF802FE0DF80E026
:103E4000DEDF5F9AFFBE8EB51F910F91FF90089540
:103E50005F9886E0D4DF5F9A82E08A95F1F7089553
:103E6000EF92FF920F931F938C01F62EEFB6F8940A
:103E7000CBDFEEDF5F9882E0C2DF812FC0DF802FD3
:103E8000BEDF8F2DBCDF5F9AEFBE1F910F91FF90B9
:103E9000EF900895DF92EF92FF920F931F93CF93CD
:103EA000DF93EC017B018A01DFB6F894ADDFD0DF50
:103EB0005F9882E0A4DF8D2FA2DF8C2FA0DFF701B7
:103EC00081917F019CDF2196CE018F719070892BAB
:103ED00019F00150104099F75F9A0115110531F75B
:103EE000DFBEDF91CF911F910F91FF90EF90DF9098
:103EF0000895DF92EF92FF920F931F93CF93DF937A
:103F00008C017B01EA01DFB6F8947EDF5F9883E0E5
:103F100076DF812F74DF802F72DF07C080E06FDFD4
:103F20008EB5F70181937F0121972097B9F75F9AAA
:103F3000DFBEC701DF91CF911F910F91FF90EF90EE
:103F4000DF900895CF93DF93282F342F662311F449
:103F500080E033C0862F90E0019760E270E00E941D
:103F6000602B6F5F41E050E026C0922F9770822F48
:103F7000869586958695A82FB0E0FD01E856FB4F03
:103F8000E081892F332349F0EA0102C0CC0FDD1F05
:103F90008A95E2F7CE018E2B09C0EA0102C0CC0F50
:103FA000DD1F8A95E2F7CE0180958E23A856BB4F80
:103FB0008C932F5F61506623C1F6DF91CF910895F6
:103FC00090E0019760E270E00E94602B6F5F40E03C
:103FD00031E0E32FE695E695E695F0E0E856FB4FF5
:103FE000808190E0232F277002C0959587952A95B0
:103FF000E2F780FD07C04F5F461729F4832F841B2B
:104000008F5F089540E03F3F11F03F5FE2CF8AB5F8
:1040100080648ABD80E008950F931F93182F21E1DB
:1040200030E0F999FECFF999FECF32BD21BDF89A63
:1040300080B5811701F50FB7F894F999FECFF9997A
:10404000FECF1FBA32BD21BD10BC0FB6F894FA9A4C
:10405000F99A0FBE812F90E025E0880F991F2A95CD
:10406000E1F74396DEDE682F6C5E812F40E06ADF69
:104070000FBF81E008C081E02031380719F02F5FC1
:104080003F4FCFCF80E01F910F910895782F20E010
:1040900031E001C09A01F999FECFA9014150504089
:1040A000CA018F5E9F4F92BD81BDF89A80B588236B
:1040B00089F381E02030380711F480E00895F99900
:1040C000FECFF999FECF1FBA2F5E3F4F32BD21BD03
:1040D00070BD0FB6F894FA9AF99A0FBE872F41E097
:1040E00031DF81E008951F93CF93DF9380E2E8E909
:1040F000F4E0DF011D928A95E9F781E0809398044E
:10410000C1E1D0E0F999FECFF999FECFD2BDC1BD92
:10411000F89A10B5112379F0812F90E035E0880FDF
:10412000991F3A95E1F743967CDE682F6C5E19F093
:10413000812F41E007DF2196B1E0C131DB0711F7A4
:10414000DF91CF911F9108951F931FB7F89420E03E
:1041500030E0822FF999FECFF999FECF1FBA90E097
:104160008F5E9F4F92BD81BD10BC0FB6F894FA9A36
:10417000F99A0FBE2F5F3F4F81E02030380749F793
:10418000B2DF1FBF1F91089580E0089585E29BE094
:1041900060E00E947C0B882369F0F89428E088E1B5
:1041A00090E00FB6F894A895809360000FBE20931E
:1041B0006000FFCF08958FD882E060E86BD884E17B
:1041C00060E080D889E59CE007D980E061E07AD89A
:1041D00087E69CE001D981E060E05CD880E2E0D82D
:1041E00088EF99E0F9D880E2DBD885E599E0F4D84A
:1041F00080E062E067D882E060E84CD884E69CE02A
:10420000EBD881E060E046D880E2CAD88EE699E03B
:10421000E3D882E060E83ED880E063E053D881E6EE
:104220009CE0DAD882E060E035D880E2B9D889E550
:1042300099E0D2D880E2B4D885E699E0CDD88DE572
:104240009BE060E070E00E94CC0A0E9422198091FD
:10425000C3029091C4028050904809F0ACCF80E036
:104260000895EF92FF920F931F93CF93DF9333D86C
:1042700085E060E027D882E060E80CD88BE69CE01F
:10428000ABD883E061E01ED801E0C0E0D0E081E07F
:10429000E82EF12CCE016FE370E00E944C2B892BAD
:1042A000B1F4209731F080E00BD88FEF09D88FEF71
:1042B00007D8102F1F5F83E0602F04D88FEF00D83E
:1042C0008FEF0E94601980E00E946019012FCE01DB
:1042D00068E070E00E94602BDC01CB01970102C016
:1042E000220F331FAA95E2F788569B4FFC0180816D
:1042F00090E0822393238217930711F48CE901C085
:1043000080E80E9460192196F1E0C030DF0709F0D3
:10431000C1CF80E00E9460198FEF0E9460198FEF7B
:104320000E94601982E06EE70E944A1980E065E011
:104330000E9462198DE59BE04FD80E94221980E00F
:10434000DF91CF911F910F91FF90EF90089582958B
:10435000807F682BEEEAFCE0E60FF11DE4918E2FE2
:1043600008958295807F682B8EEA9CE0FC01E60F21
:10437000F11DE4914295407FE42B8E0F911DFC01CD
:1043800084910895EEEAFDE0E80FF11DE4918E2F8F
:104390000895EEEBFDE0E80FF11DE4918E2F0895F6
:1043A0001F93182F613071F0862FECDF9FE0981B70
:1043B000892FEFDF1295107F182BE12FF0E0E255E7
:1043C000F34F84911F910895982F9295907F982B89
:1043D000EEEAFCE0E90FF11DE4918E2F08952F9293
:1043E0003F924F925F926F927F928F929F92AF9285
:1043F000BF92CF92DF92EF92FF920F931F93DF93C2
:10440000CF93CDB7DEB728970FB6F894DEBF0FBEB7
:10441000CDBF3C017B836A83842E1B01198225C199
:10442000D3011D91B887AF83B981BB2349F4EFE075
:10443000DE2ED122E12EE2947FE0E722EBEF0AC0EC
:10444000D12ED2946FE0D622D3011196EC90BFE02A
:10445000EB22ECEF8E0E8FE06D2D79DFF82E87E0EA
:104460006E2D75DF182F6E2D6D2589E070DFA82E5B
:10447000A29450EFA5221F25A12A85E06D2D67DFAC
:10448000C82E83E06E2D63DF182F88E06D2D5FDF6F
:10449000082F8CE06E2D5BDF08270295007F1C251E
:1044A000012B8AE06E2D53DF182F8D2D67E04FDF33
:1044B000E8268CE06E2D4BDF982E929440EF9422EC
:1044C0001F25912A4F8058840894411C511CBB24FD
:1044D000B394AF81B8858C91B981BB2339F4282F6F
:1044E0002F70982F92959F70320107C0282F229528
:1044F0002F703201F20190819F703FE0F32EFA207D
:10450000F22687E06F2D9E8322DF1A2D12951F70F1
:1045100018279E811927812F67E019DFE82E8F2D3C
:1045200069E015DFD82E812F69E011DFA82E8F2DCD
:1045300063E00DDF902F907FA826A29480EFA82241
:10454000A9260F70DE240D25A02A8F2D6CE0FFDE3A
:10455000E82E812F63E0FBDEC82E812F6CE0F7DEB2
:10456000D82E8F2D6AE0F3DE992D907F082F0D2530
:104570000295007F0927FFE09F22CE249C24092971
:10458000812F6AE0E4DE9D2C929410EF9122E826C0
:104590009E28B3940894411C511C4F8158854F5F4D
:1045A0005F4F58874F8354E0B51609F092CFD3017F
:1045B0001C91B981BB2319F4612F6F7006C0612F64
:1045C00062956F700894611C711CE981F1E0EF271E
:1045D000E9831A2D1F701627812F67E0B8DEB82EE9
:1045E000812F69E0B4DEE82E812F6CE0B0DEC82EAA
:1045F000812F63E0ACDE582EDD24812F6AE0A7DE38
:10460000202F30E02F703070FF242E253F25B4E09E
:10461000220F331FBA95E1F7A294AFE0AA22AB2490
:10462000A22AD101AC92292D30E02F7030702C25B8
:104630003D25F4E0220F331FFA95E1F702950F7044
:104640000525022B11960C9311979294EFE09E2270
:10465000982674E0CC0CDD1C7A95E1F79C28129624
:104660009C92E3E0F0E02E0E3F1E522CFA815F1A7E
:1046700024E0281508F4D4CE882D90E04981840FD9
:10468000911D892B09F429C18820E1F0D3011D91E6
:10469000B887AF83482D4150B981BB2341F46FE007
:1046A000D62ED122E12EE2945FE0E52209C0D12E80
:1046B000D2943FE0D322D3011196EC90BFE0EB22DD
:1046C000B42E0BC0F301D190F887EF83D2942FE082
:1046D000D222BB24BA94EE2419828FE06D2D37DEEE
:1046E000F82E87E06E2D33DE182F6E2D6D2589E0B4
:1046F0002EDE982E929490EF99221F25912A85E024
:104700006D2D25DEC82E83E06E2D21DE182F88E06A
:104710006D2D1DDEA82E8CE06E2D19DEA826A2942C
:1047200080EFA8221C25A12A8AE06E2D10DE182F0A
:104730008D2D67E00CDEE8268CE06E2D08DE882EDD
:10474000829400EF80221F25812A77247394BB2056
:10475000C9F0EF81F88521914B2D415059815523A6
:1047600041F4322F3F70022F02950F70F887EF83CC
:1047700007C0322F32953F70F887EF8300810F70AA
:10478000B42E0FC08981882319F430E000E009C0FD
:10479000AF81B8853D91B887AF8332953F7000E017
:1047A0001982BFE0FB2EF920F32687E06F2DCFDDC5
:1047B000192D12951F7018271027812F67E0C7DD6C
:1047C000E82E8F2D69E0C3DDD82E812F69E0BFDD93
:1047D000982E8F2D63E0BBDD9A2D907F98269294C2
:1047E000A0EF9A229926BFE0AB22DE24AD249A28BE
:1047F0008F2D6CE0ACDDE82E812F63E0A8DDC82EA4
:10480000812F6CE0A4DDD82E8F2D6AE0A0DD982DDD
:10481000907FA82EAD24A294F0EFAF22A926EFE05E
:104820008E22CE248C24A828812F6AE090DD8D2C46
:104830008294E0EF8E22E8268E287394F4E07F16AF
:1048400009F085CF7FE0D72ED9208D2D67E07FDD61
:10485000B82E8D2D69E07BDD182F8D2D6CE077DD76
:10486000E82E8D2D63E073DDC82EFF248D2D6AE0C8
:104870006EDD2A2D30E02F703070412F50E024275C
:10488000352764E0220F331F6A95E1F792945FE0C9
:1048900095229B24922AF1019192282D30E02F70CD
:1048A00030702E253F2544E0220F331F4A95E1F753
:1048B000A2943FE0A322AC24A22AD1011196AC928B
:1048C00082949FE08922882684E0EE0CFF1C8A9562
:1048D000E1F78E288182B3E05B0E852D28960FB616
:1048E000F894DEBF0FBECDBFCF91DF911F910F9126
:1048F000FF90EF90DF90CF90BF90AF909F908F9000
:104900007F906F905F904F903F902F9008952F92DF
:104910003F924F925F926F927F928F929F92AF924F
:10492000BF92CF92DF92EF92FF920F931F93DF938C
:10493000CF9300D00F92CDB7DEB72B011C01882496
:10494000D101ED913D01FE2EFFE0FF22CE2EC2945B
:10495000BFE0CB228FE06F2DFADCD82E87E06C2DE4
:10496000F6DC182F6C2D6F2589E0F1DCA82EA294BF
:10497000A0EFAA221D25A12A85E06F2DE8DCE82EF4
:1049800083E06C2DE4DC182F88E06F2DE0DC082F2D
:104990008CE06C2DDCDC08270295007F1E25012BA6
:1049A0008AE06C2DD4DC182F8F2D67E0D0DCC82670
:1049B0008CE06C2DCCDC982E9294F0EF9F221D257C
:1049C000912A44E050E0240E351ED3011D913D0193
:1049D000F12EFA24BFE0FB2287E06F2DB8DC1295A0
:1049E0001F701827A294EFE0AE221A25812F67E0EE
:1049F000AEDCE82E8F2D69E0AADCD82E812F69E08D
:104A0000A6DCA82E8F2D63E0A2DC902F907FA82635
:104A1000A29470EFA722A9260F70DE240D25A02AEC
:104A20008F2D6CE094DCE82E812F63E090DCC82EA3
:104A3000812F6CE08CDCD82E8F2D6AE088DC992DDC
:104A4000907F082F0D250295007F0927EFE09E2219
:104A5000CE249C240929812F6AE079DC9D2C929434
:104A600060EF9622E8269E286214730409F0ADCF09
:104A70005FE0D52EDA208D2D67E069DCB82E8D2D14
:104A800069E065DC182F8D2D6CE061DCE82E8D2D42
:104A900063E05DDCC82EFF248D2D6AE058DC202FFA
:104AA00030E02F703070412F50E02427352744E04C
:104AB000220F331F4A95E1F7A2943FE0A322AB24D3
:104AC000A22AD201AC92292D30E02F7030702E2511
:104AD0003F2594E0220F331F9A95E1F702950F705E
:104AE0000C25022B11960C93119792941FE09122A2
:104AF0009826F4E0EE0CFF1CFA95E1F79E2812963A
:104B00009C928394B5E08B1631F0E3E0F0E04E0E1A
:104B10005F1E130115CF0F900F900F90CF91DF9173
:104B20001F910F91FF90EF90DF90CF90BF90AF90CB
:104B30009F908F907F906F905F904F903F902F90BD
:104B400008953F924F925F926F927F928F929F92C1
:104B5000AF92BF92CF92DF92EF92FF920F931F938B
:104B6000CF93DF936C013B01542EE901402EEE24DC
:104B70003324339449010894811C911C22E0A22E15
:104B8000B12CAC0EBD1EE41410F0FF2410C0F601D1
:104B90001081552021F49FE0F92EF12207C0F12E5B
:104BA000F2948FE0F8220894C11CD11C5324088190
:104BB000802F8F7062E0CBDB182F802F82958F7053
:104BC00064E0C5DB8F258295807F1F25812B88833C
:104BD000F4010081802F8F7068E0B9DB182F802FDF
:104BE00082958F7063E0B3DB8F258295807F1F25D0
:104BF000812BF4018083F5011081812F8F7066E095
:104C0000A6DB082F812F82958F706CE0A0DB8F25AB
:104C10008295807FF026F82AF501F082E394F9E08E
:104C2000EF1609F0B0CFDD24EE24CC24C394F301B9
:104C30001081DD2021F40FE0F02EF12207C0F12ECB
:104C4000F2941FE0F1220894611C711C0881802FEE
:104C50008F7062E07CDB182F802F82958F7064E06C
:104C600076DB8F258295807F1F25812B8883F40139
:104C70000081802F8F7068E06ADB182F802F82956B
:104C80008F7063E064DB8F258295807F1F25812BE9
:104C9000F4018083F5011081812F8F7066E057DB6E
:104CA000082F812F82958F706CE051DB9F2D982704
:104CB0009295907FF0269F29F5019083E394F6E08A
:104CC000EF1611F0DC24B3CF8981982B8881892BD2
:104CD000DF91CF911F910F91FF90EF90DF90CF90D8
:104CE000BF90AF909F908F907F906F905F904F900C
:104CF0003F9008952F923F924F925F926F927F92D2
:104D00008F929F92AF92BF92CF92DF92EF92FF92DB
:104D10000F931F93CF93DF93EC012B01E880CE2CF0
:104D2000C294BFE0CB2219818C2D90E02E2D30E073
:104D30002F703070822B932B212F30E02F7030702A
:104D4000822B932B892B11F480E0DDC0AFE08A2EFB
:104D50008122DA80FFE06F2E6D20882D662DF7DA34
:104D6000A82E912E9294EFE09E22892D2DDBA8266D
:104D70008C2D692DECDA382E882D26DB282E38264E
:104D80008C2D662DE4DAF82E882D692DE0DA082FB7
:104D90007FE0B72EBE208B2D6A2DD9DA182F882DF3
:104DA000632DD5DA782E802F8F256C2DD0DA7126E1
:104DB000782609F475C08C2D6A2DC9DAE82E8C2D61
:104DC00003DB0D2D02950F70602FC1DA182F8B2D8C
:104DD000692D462DC6DAF82E8B2D682D402FC1DAAD
:104DE000082F822D692DB3DA1E251F251027812754
:104DF000672DD6DAF20181936F0109816FE0962E5B
:104E00009022892D6A2DA3DA882EF880AF2CA294E7
:104E10005FE0A52202950F70BA804FE0E42EEB20F0
:104E20008A2D602F4E2D9DDA182FFFE0FF226B2C6C
:104E300062943FE063228F2D602F462D92DAB82EC8
:104E40008E2DC2DA6F2D83DA082F8A2D692D462D1B
:104E500088DA18251B2510278127672DA1DAF20192
:104E600081831A81812F82958F70632D70DAF82EDD
:104E7000812F8F70A9DA682F888182958F7067DA09
:104E8000082F198112951F70812F9EDA612F5FDA2A
:104E90000F258027672D84DAF601818383E033C0F4
:104EA000AA2019F1862D90DA182F8D2D82958F70FA
:104EB000692D4DDA81276A2D73DAF2018083F9803A
:104EC0001A81612F62956F708F2D8F7040DA082FD5
:104ED0001F708F2D82958F70612F39DA80276A2D90
:104EE0005FDAF201818382E00EC08C2D6B2D58DADF
:104EF000182F882D6C2D54DAF2018083181711F0C9
:104F00008FEF01C081E0DF91CF911F910F91FF9052
:104F1000EF90DF90CF90BF90AF909F908F907F9059
:104F20006F905F904F903F902F900895BF92CF92D7
:104F3000DF92EF92FF920F931F93CF93DF93EC01D9
:104F40006A01623039F1633009F040C0BB24EE24BD
:104F50008E2D1FDAF82E38DA182F6F2DF8D9082F7A
:104F6000812F6881F4D9182F8F2D6981F0D91027EE
:104F700018278A81181721F4F601F1926F01B39472
:104F8000F2E0FB1520F0E3948FE0E81609F78B2D93
:104F9000835020C0EE24FF248F2DFBD9082F14DA74
:104FA000182F802F6981D3D918278881181739F4D1
:104FB000F60101936F01E394F1E0FE1520F0F39404
:104FC0008FE0F81649F78E2D825004C08881FA01CF
:104FD000808380E0DF91CF911F910F91FF90EF9040
:104FE000DF90CF90BF9008954F925F926F927F9223
:104FF0008F929F92AF92BF92CF92DF92EF92FF92E9
:105000000F931F93CF93DF933C01EB0129014230B3
:1050100009F4B8C0FC01A080433009F0E6C0FA8072
:10502000E9806E2D6F258F2D92D9982E6E2D8FD9F8
:10503000082F1881812FC8D9682F802F88D9612F18
:1050400086D9D82E6E2D61278E2D81D9612F7FD9DB
:10505000082F8F2DB9D9C82E802F6C2D78D96F2DA0
:1050600076D9B82E6F2D6127812F71D96F2D6FD909
:10507000182F8E2DA9D9082F812F602F68D96E2D5A
:1050800066D9BD24B8261FE0D12EDA208F2D6D2DD4
:105090005ED91A2D12951F70612F68278F2D57D951
:1050A000A82E802F6E2D53D9682F8A2D50D9082F06
:1050B0008E2D6D2D4CD918278E2D612F48D9882E15
:1050C0008C2D6F2D44D9682F882D41D9182FF301CD
:1050D00061816F70892D4E2D44D9102781276B2D4A
:1050E0005FD9F20181936F010881802F6DD9602F04
:1050F0002ED9682F8A2D2BD9E82EF3011081612F2C
:105100006F70802F24D912951F701827802F612F60
:105110001ED9982E1A81812F57D9612F18D9692D40
:1051200016D9F82EF30181818F70602F10D9A82E27
:105130000127812F602F0BD9682F8A2D08D9FE24D3
:105140008F256B2D2DD9F2018183F8808F2D3CD9CD
:105150006F2DFDD8682DFBD8E82E1981812F34D909
:10516000612FF5D8692DF3D8082FF126812F6F2DE7
:10517000EED8682F8A2DEBD80E2580276B2D10D9FD
:10518000F60131C01881812F1FD9D82EF9808F2DBB
:105190001BD9082F8D2D6F2DDAD8E82E802F612F87
:1051A000D6D8E826F3011081812F8F70602FCFD8D9
:1051B000082F812F82958F706F2DC9D880276E2D73
:1051C000EFD8F2018083F3011081812F8F706D2D54
:1051D000BED8082F812F82958F706881B8D880271C
:1051E0006E2DDED8F201818306C08A2D8F70688112
:1051F000D7D8F2018083DF91CF911F910F91FF905B
:10520000EF90DF90CF90BF90AF909F908F907F9066
:105210006F905F904F9008955F926F927F928F9200
:105220009F92AF92BF92CF92DF92EF92FF920F9335
:105230001F93DF93CF93CDB7DEB72C970FB6F894BB
:10524000DEBF0FBECDBF5C01842E022FDE011196A2
:10525000E0E0F1E083E001900D928150E1F7C501BB
:10526000482D7E010894E11CF11C97016ADC88231B
:1052700019F400E010E064C024E0C22ED12CCC0E62
:10528000DD1EC701B60136DD982E8FEF981619F492
:105290000FEF10E055C08E01065F1F4FC601692D4C
:1052A000A80144DE882319F00EEF10E049C097E012
:1052B000692E712C6C0E7D1EC701B801492D93011A
:1052C00093DE6801730100E010E08EE0582E34C0D8
:1052D000F601808157D8F52DF81B8F2F880D8A3065
:1052E000A8F4282F2695F701908180FF09C0F501C9
:1052F000E20FF11D9295907F80819827908306C0E0
:10530000F501E20FF11D808189278083F70140813B
:1053100098E020E030E0892F842311F00F5F1F4FC9
:1053200096952F5F3F4F24303105A9F70894E11C73
:10533000F11C0894C11CD11C8E2D8619891540F2D0
:10534000C8012C960FB6F894DEBF0FBECDBFCF912B
:10535000DF911F910F91FF90EF90DF90CF90BF9062
:10536000AF909F908F907F906F905F900895CF92B5
:10537000DF92FF920F931F93CF93DF936B018C010A
:10538000FF24C0E0D0E0B6016C0F7D1FC80140E0F3
:1053900028E042DF843040F4F80E0C5F1F4F239664
:1053A000CF30D10581F78F2DDF91CF911F910F91D4
:1053B000FF90DF90CF900895AF92BF92CF92DF928F
:1053C000EF92FF920F931F93CF93DF935C01EB015A
:1053D000142FFF24DD24EE2400E0CC24C39426C047
:1053E0008F2D90E06D2D70E0153050F06C0F7D1F0B
:1053F0008A0D9B1D402F29E00FDF1450101B0AC09F
:105400006C0F7D1F110F101B8A0D9B1D402F212F2C
:1054100003DF10E0843018F03EEFE32E09C0F00EF9
:1054200094E0F90E0C2593E0D90EE80E1123C1F695
:105430008E2DDF91CF911F910F91FF90EF90DF9014
:10544000CF90BF90AF900895CF93DF93EC01A0E091
:1054500040E050E0FA01E253F24F7491FE01E40F94
:10546000F51F8081782761E020E030E0862F8723D8
:1054700009F0AF5F660F2F5F3F4F28303105B1F75E
:105480004F5F5F4F4430510529F7A83008F4A0E082
:105490008A2FDF91CF9108958627282F22952827DC
:1054A000022E269526952025022E2695202527704A
:1054B000082E892F269507942795902D82270694EC
:1054C0002795902582270895FB01DC018D91813479
:1054D0001CF08B350CF4805E659161341CF06B35EB
:1054E0000CF4605E861B611189F3990B0895FB0132
:1054F000DC010D900020E9F7119705900D92002036
:10550000E1F70895FB01DC0105900D920020E1F721
:105510000895FB01DC014150504048F005900D9288
:105520000020C9F701C01D9241505040E0F7089596
:10553000FB01DC0102C001900D9241505040D8F7B0
:105540000895DC0101C06D9341505040E0F708958B
:10555000FB01DC018D9181341CF08B350CF4805EF5
:10556000619161341CF06B350CF4605E861B611137
:1055700089F3990B0895FB01DC0101900D92002045
:10558000E1F70895FB01DC014150504088F08D9116
:1055900081341CF08B350CF4805E619161341CF019
:1055A0006B350CF4605E861B611171F3990B0895E5
:1055B000881BFCCFFB01DC014150504048F00190BA
:1055C0000D920020C9F701C01D9241505040E0F7F4
:1055D0000895A0E0B0E0EEEEFAE2B9C07C01EB0184
:1055E0008A01690109C0CE012196F6010995F701EA
:1055F00081937F010150104001151105A1F7CDB72E
:10560000DEB7E8E0C0C0A0E0B0E0E8E0FBE29FC0A9
:10561000EC017B018A01690109C0CE012196F701E5
:1056200061917F01F60109950150104001151105A6
:10563000A1F7CDB7DEB7E8E0A6C0FB019F01E89473
:105640004230BCF04532ACF44A3029F497FB1EF4EA
:10565000909581959F4F642F77271ED0805D8A3368
:105660000CF0895D8193CB010097A9F716F45DE2F8
:1056700051931082C90100C0DC01FC01672F7191B8
:105680007723E1F7329704C07C916D937083629128
:10569000AE17BF07C8F30895AA1BBB1B51E107C093
:1056A000AA1FBB1FA617B70710F0A61BB70B881FB2
:1056B000991F5A95A9F780959095BC01CD01089541
:1056C00097FB092E07260AD077FD04D0E5DF06D028
:1056D00000201AF4709561957F4F0895F6F7909524
:1056E00081959F4F0895A1E21A2EAA1BBB1BFD01B5
:1056F0000DC0AA1FBB1FEE1FFF1FA217B307E407B1
:10570000F50720F0A21BB30BE40BF50B661F771F08
:10571000881F991F1A9469F76095709580959095E8
:105720009B01AC01BD01CF010895911108958156EF
:105730008A5108F48052855808952F923F924F92D3
:105740005F926F927F928F929F92AF92BF92CF9211
:10575000DF92EF92FF920F931F93CF93DF93CDB71A
:10576000DEB7CA1BDB0B0FB6F894DEBF0FBECDBF92
:1057700009942A88398848885F846E847D848C8463
:105780009B84AA84B984C884DF80EE80FD800C816C
:105790001B81AA81B981CE0FD11D0FB6F894DEBF4F
:0C57A0000FBECDBFED010895F894FFCFBF
:0457AC0000000000F9
:00000001FF
